:0400000057EF00F0C6
:100008002B002B002B002B002B002B002B002B0090
:100018002B002B002B002B002B002B002B002B0080
:100028002B002B002B002B002B002B002B002B0070
:100038002B002B002B00A04C2B002B002B00295051
:100048002B002B002B002B002B002B002B002B0050
:100058002B002B002B002B002B002B002B002B0040
:100068002B002B002B002B002B002B002B002B0030
:100078002B002B002B002B002B002B002B002B0020
:100088002B002B002B002B002B002B002B002B0010
:100098002B002B002B002B002B002B002B002B0000
:0A00A8002B002B00FF008DEF99F0F4
:10F65C000000000000001B1B0000181818181B1BD2
:10F66C000000030303031B1B00001B1B1B1B1B1BAA
:10F67C0000040E1F0404040400040404041F0E04FC
:10F68C00001112140B110203000E0A0E00000000F0
:10F69C000045724C754D614D654A65566553614424
:10F6AC0069000080C094D47F20417574726573200A
:10F6BC003A20204C43445F34626974735F4932438F
:10F6CC005F323032332D303931352C205541525484
:10F6DC00315F46756E6374696F6E732E682C2052A1
:10F6EC0054435F4453333233315F323032332D3035
:10F6FC00392E680D0A00204C43445F6368617273B5
:10F70C005F53706563696175785F323032332D30C9
:10F71C003832372E682C202020456570726F6D2092
:10F72C003A20456570726F6D5F323443333220641A
:10F73C0065205254430D0A00204469726563746F4E
:10F74C007279203A433A5C4D504C4142585F5072AA
:10F75C006F6A656374735C5F31384632374B343291
:10F76C005F546573745F4932435F32344333325FA5
:10F77C00323032332E580D0A0045434F2E2E2E2E8A
:10F78C000042415252455F470042415252455F444C
:10F79C00004241525245474400464C45434820489C
:10F7AC0000464C4543485F4200312F324865757224
:10F7BC00004445475245432000204C4344203478B4
:10F7CC0032302063617273202B20525443207375A6
:10F7DC0072206275732049324331204857203A20F9
:10F7EC005243333D53434C2C5243343D5344410D0F
:10F7FC000A00204120696E636C7572653A202044C2
:10F80C0069616C6F6775655F4F7065726174657562
:10F81C00725F50435F323032332D303932342E69BF
:10F82C006E63200D0A0D0A002050494331384632D0
:10F83C00374B3432202B203378204F5753204453EE
:10F84C00313842323020737572205241302C524183
:10F85C00312C5241320D0A002050726F6A6563746C
:10F86C00203A20205F31384632374B34325F5465B2
:10F87C0073745F4932435F32344333325F32303218
:10F88C00330D0A00204861726477617265203A205A
:10F89C0042726561626F61726420262042617365F9
:10F8AC002031384632374B3432200D0A0020524179
:10F8BC00343D6C65642C20205243363D5458205501
:10F8CC0041525431205243373D52582055415254E5
:10F8DC000D0A0020536F75726365203A20206D610C
:10F8EC00696E2E63202C20726576203A5F3230329E
:10F8FC00332D313031320D0A0020436F6E6669674B
:10F90C002020496E7465726E616C20466F736320A3
:10F91C0036344D487A0D0A0020202020202020204B
:10F92C002020202020202020202020200053657023
:10F93C0074656D627265200044696D616E63686503
:10F94C00200056656E647265646920004D657263B3
:10F95C00726564692000446563656D6272652000A0
:10F96C004E6F76656D62726520004F63746F6272C4
:10F97C006520004A75696C6C65742000466576726A
:10F98C0069657220004A616E766965722000536168
:10F99C006D656469200065727265757220004A6538
:10F9AC0075646920004D6172646920004C756E6449
:10F9BC006920004572726F722000417672696C206A
:10F9CC0000416F757420004A75696E20004D61729C
:10F9DC007320004D61692000200D0A0020200020BA
:10F9EC0056657273696F6E20323032332D3130317F
:10F9FC00320D0A2050726F6772616D6D65206465FF
:10FA0C002054657374207375722045656570726F30
:10FA1C006D203234433332206475206D6F64756C05
:10FA2C006520525443204453333233310D0A202085
:10FA3C0028206574206176656320204C434420495E
:10FA4C0032432050434638353734290D0A002045BF
:10FA5C0074617420746D705B5D2C20257320617053
:10FA6C007265732065637269747572652064616E6A
:10FA7C007320656570726F6D200D0A20746D705B5C
:10FA8C00305D3D2564202020305825303258202010
:10FA9C00746D705B315D3D2564202030582530320B
:10FAAC0058200D0A002065783A20553B32383B30FF
:10FABC00383B32333B31383B31343B30313B232004
:10FACC0020706F757220323820416F75742032307F
:10FADC003233202C2031384831342C4C756E64690B
:10FAEC00200D0A0020484D3D78783A797920207312
:10FAFC006574204865757265287878294D696E752E
:10FB0C00746573287979292053414E53206C6965AB
:10FB1C006E206176656320525443202120200D0A0B
:10FB2C000020553B32343B30383B31373B31383B8E
:10FB3C0033363B3034232020706F757220323420E2
:10FB4C00416F7574203230313720203138483336CC
:10FB5C002030343D4A657564690D0A0D0A00204C4D
:10FB6C0065637475726520646520382062797465EC
:10FB7C00732C20646570756973206C2761647265E1
:10FB8C007373652033323020456570726F6D20328F
:10FB9C00344333320D0A000D0A2052617070656CCB
:10FBAC0020666F726D617420646520636465203A11
:10FBBC002022553B4A4A3B4D4D3B41413B48483B3B
:10FBCC004D4D3B6A533B2322200D0A0020456372A6
:10FBDC0069747572652064616E7320456570726F0F
:10FBEC006D20323443333220E0206C27616472651F
:10FBFC0073736520333230206465203A0D0A00207F
:10FC0C004C434420426C65752073757220427265BA
:10FC1C006164626F617264202061647265737365E4
:10FC2C0020376269747320203078323720210D0A16
:10FC3C0000204020646563696D616C202325347558
:10FC4C002020736F697420404465766963652037A2
:10FC5C0062697473203D20305825303258200020C2
:10FC6C005052473D787820202050726F6772616D3A
:10FC7C006D6520656E20636F7572732078783D20FA
:10FC8C00303020E020313120200D0A0020457461F5
:10FC9C0074204272756C657572204252553D30204D
:10FCAC006F7520312028706F757220746573742005
:10FCBC006F6E6C7929200D0A002053657175656E85
:10FCCC006365206427496E6974204C434420347862
:10FCDC003230207669612049324331205043463816
:10FCEC00353734203A00204368617267656D656E64
:10FCFC0074206361726163746572657320537065FF
:10FD0C0063696175782020656E20434752414D0D23
:10FD1C000A0020746D705B305D3D253364203078B3
:10FD2C0025303258202C20746D705B315D3D2533AD
:10FD3C00642020307825303258200D0A00204241B2
:10FD4C00563D782020206D6F64652042617661728B
:10FD5C0064206176656320783D3020E020392020D6
:10FD6C000D0A0020546573742070726573656E63A0
:10FD7C0065206465766963657320737572204275BE
:10FD8C007320493243310D0A0020736920484D3DE0
:10FD9C0030303A30302020757361676520525443FF
:10FDAC002072E96163746976E90D0A000D0A204E30
:10FDBC0065772074696D652020486F75723D253319
:10FDCC0064204D696E753D25336420200D0A00209A
:10FDDC0023312041637469766520736F7274696591
:10FDEC0020525443205351573D31487A202E2E2E09
:10FDFC00000D0A45727265757220737572204A6F18
:10FE0C0075722053656D61696E65206A532E200DE5
:10FE1C000A002061647265737365204C43443D2075
:10FE2C00256420736F697420305825303258200DAA
:10FE3C000A00456570726F6D2032344C43787878C7
:10FE4C00203235366B206F75203531324B00205007
:10FE5C0043463837353420666F72204C4344203289
:10FE6C00783136636172730020496E69745F493270
:10FE7C0043282920E0203130304B687A3B0D0A00B2
:10FE8C004563726974757265204453333233312E75
:10FE9C002E2E204F4B0D0A00205265736574204D99
:10FEAC004355203A20526573657420200D0A000DCD
:10FEBC000A20526573657420766F6C6F6E7461697D
:10FECC007265200D0A0020526573756C7461742084
:10FEDC006C6563747572653A200D0A000D0A204832
:10FEEC00656C7020436F6D6D616E646573203A0DA7
:10FEFC000A00386361727320434752414D20202021
:10FF0C002020202020200056657273696F6E2042DD
:10FF1C0072656164626F617264202100456372696D
:10FF2C007475726520456570726F6D32344333326F
:10FF3C000050434638353734412038626974732099
:10FF4C00492F4F00204D414A20525443207669617D
:10FF5C00203A200D0A004C434420323131392032F2
:10FF6C0078313663617273004E625F426F75636CF9
:10FF7C0065733A20253564200050434638353734B4
:10FF8C0020386269747320494F00454550524F4DDB
:10FF9C00203531326279746573004C656374757207
:10FFAC006520323443333220000D0A204D414A2063
:10FFBC00525443200D0A004F4C45442053534431B6
:10FFCC00333036006E6F6E20726563656E73E900B8
:10FFDC0052544320445333323331002048656C7003
:10FFEC00200D0A0052656375203A006C6C7300207A
:04FFFC002E310000A2
:020000040001F9
:10000000600E3901D96F000EDB6F000EDD6F080E38
:10001000DF6F000EDE6F090E0101EA6F1E0EE96F41
:10002000E40EE82EFED7E92FFCD7EA2FFAD700F02E
:10003000D29E000E3A01456F000E466F000E476FCC
:10004000000E656F000E666F000E676F000E556F35
:10005000000E566F3901909FA29F928FA3919381BA
:10006000D2909191A09FA19100019E9F2DEC98F0BC
:10007000000E5C6E000E5B6E000E5B24D96E030EEC
:100080005C20DA6E000EDF6E5B4A5C2A5C5009E190
:10009000800E5B5CD8A04FEF80F051EF80F03CEF1A
:1000A00080F0000E5C6E000E5B6E800E5B24D96EDD
:1000B000020E5C20DA6E000EDF6E5B4A5C2A5C503A
:1000C00009E1800E5B5CD8A068EF80F06AEF80F0F9
:1000D00055EF80F0000E5C6E000E5B6E000E5B2430
:1000E000D96E020E5C20DA6E000EDF6E5B4A5C2A6F
:1000F0005C5009E17F0E5B5CD8A081EF80F083EF5C
:1001000080F06EEF80F0000E5C6E000E5B6EB80E3D
:100110005B24D96E000E5C20DA6E000EDF6E5B4A47
:100120005C2A5C5009E1090E5B5CD8A09AEF80F074
:100130009CEF80F087EF80F0000E0001826F030ECD
:10014000836F020E8DEC9DF032EC9EF0090E0101E2
:10015000EA6F1E0EE96FE40EE82EFED7E92FFCD7FA
:10016000EA2FFAD700F0FDEC9FF0EB0E026EF90ECD
:10017000036E62EC9DF0740E026EFE0E036E62EC76
:100180009DF073ECA0F0090E0101EA6F1E0EE96FFD
:10019000E40EE82EFED7E92FFCD7EA2FFAD700F0BD
:1001A0006F0E026EFD0E036E62EC9DF0EEEC8BF0B6
:1001B0003D01739F7599738FFDEC9FF0DB0E026E0E
:1001C000FD0E036E62EC9DF0B80E0001926F000E02
:1001D000936F400EB86F0E0E026E92C003F093C084
:1001E00004F0010E056E680E33EC9DF09E0E026E5B
:1001F000FE0E036E62EC9DF0090E0101EA6F1E0E09
:10020000E96FE40EE82EFED7E92FFCD7EA2FFAD7E4
:1002100000F0FDEC9FF0270E5D6E000E0001F56F03
:10022000140EF46F000ED96F020EDA6F1E0EDB6F24
:10023000FE0EDC6F5DC0DDF0DE6B5DC0DFF0E06BFD
:10024000E0EC9DF0000E026E020E036ECCEC97F017
:10025000C50E026EFC0E036E62EC9DF0ABEC92F0EC
:10026000FDEC9FF0010E25EC9AF00B0E026EFC0ED9
:10027000036E62EC9DF0010E0D6E130E0E6EFF0EFE
:100280000F6E010E8FECA0F0020E8DEC9DF0F20EC1
:10029000026EFC0E036E62EC9DF0000E096E000E05
:1002A000086E0CEC92F0010E0D6EFE0E0E6EFE0E40
:1002B0000F6E020E8FECA0F0000E5C6E000E5B6EF7
:1002C000000E096E020E086E0D0E5B240A6E000E03
:1002D0005C200B6E5BC00CF06AEC97F05B4A5C2A0A
:1002E0005C5009E1080E5B5CD8A079EF81F07BEFF0
:1002F00081F060EF81F0020E8DEC9DF0000E0D6E2E
:10030000040E0C6E40EC96F0000E0D6E030E0C6E9B
:1003100040EC96F0000E46EC93F0030E0D6EE00EEE
:100320000E6E010E0F6E030E82ECA0F0030E0D6E2A
:10033000F60E0E6E000E0F6E040E82ECA0F0FDECB9
:100340009FF0020E8DEC9DF0DDEC9EF03901909F48
:10035000000E3A01866F000E556F000E566F000EAC
:10036000576F3901A09F00019E9F3901A191919182
:10037000D29E270E5D6E010E25EC9AF0010E0D6ED9
:10038000280E0E6EFF0E0F6E010E8FECA0F0020E07
:100390008DEC9DF0310E0001B86F320EB96F330E47
:1003A000BA6F340EBB6F350EBC6F360EBD6F370E95
:1003B000BE6F000EBF6F000EC06F000EC16FB80E93
:1003C000926F000E936FD80E026EFB0E036E62ECFE
:1003D0009DF092C002F093C003F0CCEC97F0FDECDE
:1003E0009FF0570E5D6EBA86010E036E400E026ED0
:1003F000B80E046E000E056E080E066E5D50FAEC27
:100400009AF0BA96B80E0001926F000E936F000E2C
:10041000C16F270E5D6E010E0D6E92C00EF093C07F
:100420000FF0020E82ECA0F0B80E0001926F000EE9
:10043000936F000ED96F020EDA6F5A0EDB6FFA0E51
:10044000DC6F92C0DDF093C0DEF0B8C0DFF0E06B8F
:10045000B8C0E1F0E26BB9C0E3F0E46BB9C0E5F01D
:10046000E66BE0EC9DF0000E026E020E036ECCEC2B
:1004700097F0FDEC9FF0020E8DEC9DF06A0E026E7F
:10048000FB0E036E62EC9DF0000E5C6E000E5B6E68
:10049000B80E5B24D96E000E5C20DA6E000EDF6EA3
:1004A0005B4A5C2A5C5009E1090E5B5CD8A05BEFFB
:1004B00082F05DEF82F048EF82F0B80E0001926F9B
:1004C000000E936F570E5D6EBA86010E036E400EDE
:1004D000026EB80E046E000E056E080E066E5D50BC
:1004E0006FEC9AF0BA96B80E0001926F000E936FFF
:1004F000D20E026EFE0E036E62EC9DF092C002F010
:1005000093C003F0CCEC97F0FDEC9FF0000E0001DF
:10051000D96F020EDA6F1E0EDB6FFD0EDC6FB8C0F6
:10052000DDF0DE6BB8C0DFF0E06BB9C0E1F0E26B8C
:10053000B9C0E3F0E46BE0EC9DF0000E026E020E39
:10054000036ECCEC97F0030E8DEC9DF0270E5D6EE4
:10055000010E25EC9AF0010E0D6EA60E0E6EFF0E2A
:100560000F6E010E8FECA0F0010E8DEC9DF0010ED0
:100570000D6E92C00EF093C00FF0020E82ECA0F050
:10058000000E0001876F000E866F6AC06FF16BC0AE
:1005900070F1010E46EC93F0010E0D6EE00E0E6E42
:1005A000010E0F6E030E82ECA0F00C0E0D6EF60E17
:1005B0000E6E000E0F6E030E82ECA0F0FDEC9FF0AD
:1005C000000E0001D96F020EDA6F740EDB6FFF0EA2
:1005D000DC6F86C0DDF087C0DEF0E0EC9DF0010E40
:1005E0000D6E000E0E6E020E0F6E040E82ECA0F069
:1005F000020E8DEC9DF0B6EC9BF0020E8DEC9DF0A2
:100600000001B605D8A407EF83F009EF83F09CEF53
:1006100085F0F00E026EFF0E036E62EC9DF0800E10
:10062000026E020E036ECCEC97F0FDEC9FF0800E94
:10063000596E020E5A6E600067F1D9FF60006BF1CF
:10064000DAFF550EDE18D8A428EF83F02AEF83F0E6
:1006500067EF83F020EE01F05950D9265A50DA2284
:100660003B0EDE18D8A437EF83F039EF83F067EF45
:1006700083F020EE13F05950D9265A50DA223B0E5F
:10068000DE18D8A446EF83F048EF83F067EF83F0DD
:1006900000019F51D8A44FEF83F051EF83F067EF33
:1006A00083F0B50E026EFF0E036E62EC9DF0800EBD
:1006B000026E020E036ECCEC97F0FDEC9FF01EEC88
:1006C0008EF0FDEC9FF0000E596E000E5A6E600029
:1006D00067F1D9FF60006BF1DAFF480EDE18D8A48D
:1006E00074EF83F076EF83F0EBEF83F020EE01F010
:1006F0005950D9265A50DA22650EDE18D8A483EF55
:1007000083F085EF83F0EBEF83F020EE02F0595099
:10071000D9265A50DA226C0EDE18D8A492EF83F054
:1007200094EF83F0EBEF83F020EE03F05950D926DD
:100730005A50DA22700EDE18D8A4A1EF83F0A3EF8E
:1007400083F0EBEF83F0E80E026EFE0E036E62ECB8
:100750009DF0500E026EFF0E036E62EC9DF0B10E26
:10076000026EFA0E036E62EC9DF06B0E026EFC0ED2
:10077000036E62EC9DF0490E026EFD0E036E62EC9C
:100780009DF0F00E026EFA0E036E62EC9DF0950E77
:10079000026EFD0E036E62EC9DF0980E026EFC0E72
:1007A000036E62EC9DF0A40E026EFE0E036E62EC10
:1007B0009DF0E70E026EFF0E036E62EC9DF0800E60
:1007C000026E020E036ECCEC97F0FDEC9FF0000E73
:1007D000596E000E5A6E600067F1D9FF60006BF130
:1007E000DAFF420EDE18D8A4F8EF83F0FAEF83F0B8
:1007F00047EF84F020EE01F05950D9265A50DA2202
:10080000410EDE18D8A407EF84F009EF84F047EF1B
:1008100084F020EE02F05950D9265A50DA22560EB2
:10082000DE18D8A416EF84F018EF84F047EF84F0B8
:1008300020EE03F05950D9265A50DA223D0EDE1828
:10084000D8A425EF84F027EF84F047EF84F020EE62
:1008500004F05950D9265A50DA22DF500001A26F15
:100860002F0EA26536EF84F038EF84F043EF84F06A
:100870003A0EA2613EEF84F040EF84F043EF84F043
:10088000A251D00FB36F000E596E000E5A6E600069
:1008900067F1D9FF60006BF1DAFF480EDE18D8A4CB
:1008A00054EF84F056EF84F024EF85F020EE01F051
:1008B0005950D9265A50DA224D0EDE18D8A463EFCB
:1008C00084F065EF84F024EF85F020EE02F05950BB
:1008D000D9265A50DA223D0EDE18D8A472EF84F0E1
:1008E00074EF84F024EF85F020EE05F05950D926FE
:1008F0005A50DA223A0EDE18D8A481EF84F083EF42
:1009000084F024EF85F020EE03F05950D9265A5098
:10091000DA22DF500001A26FA2C0F6F0A251D00F80
:10092000A26FA2510A0D6F00CCFF8EF06F00D0FFB6
:100930008FF020EE04F05950D9265A50DA22DF50B9
:10094000A26FA2C0F7F0A251D00FA26FA2518E25C4
:100950008E6F000E8F218F6F8F5107E1180E8E5D05
:10096000D8B0B5EF84F0B7EF84F0ECEF84F020EE70
:1009700006F05950D9265A50DA22DF50A26FA2C091
:10098000F9F0A251D00FA26FA2510A0D6F00CCFF57
:100990008AF06F00D0FF8BF020EE07F05950D92677
:1009A0005A50DA22DF50A26FA2C0FAF0A251D00F43
:1009B000A26FA2518A258A6F000E8B218B6F8F51F7
:1009C00007E13C0E8E5DD8B0E8EF84F0EAEF84F0EA
:1009D000ECEF84F08AC0A8F08E518F11D8A4F3EF09
:1009E00084F0F5EF84F002EF85F08A518B11D8A4E2
:1009F000FCEF84F0FEEF84F002EF85F0000E9F6FB5
:100A000020EF85F08EC0AAF08AC0A8F0010E9F6F7B
:100A1000000EA96F000ED96F020EDA6FB80EDB6FF1
:100A2000FD0EDC6FAAC0DDF0DE6BA8C0DFF0E06B6E
:100A3000E0EC9DF0000E026E020E036ECCEC97F01F
:100A4000000E596E000E5A6E600067F1D9FF60000B
:100A50006BF1DAFF520EDE18D8A431EF85F033EFD8
:100A600085F09CEF85F020EE01F05950D9265A50C0
:100A7000DA22450EDE18D8A440EF85F042EF85F06B
:100A80009CEF85F020EE02F05950D9265A50DA2218
:100A9000530EDE18D8A44FEF85F051EF85F09CEF90
:100AA00085F020EE03F05950D9265A50DA22450E2F
:100AB000DE18D8A45EEF85F060EF85F09CEF85F03E
:100AC00020EE04F05950D9265A50DA22540EDE187E
:100AD000D8A46DEF85F06FEF85F09CEF85F059C0DD
:100AE00002F05AC003F057EC9FF0050E02180310F5
:100AF000D8A47DEF85F07FEF85F098EF85F0000EAC
:100B00000001D96F020EDA6FBB0EDB6FFE0EDC6FD9
:100B1000E0EC9DF0000E026E020E036ECCEC97F03E
:100B2000000E596E000E5A6E040E8DEC9DF0FF0003
:100B3000000E596E000E5A6EBA780001864B872B54
:100B4000C5EF82F057EF00F060000FF1D9FF6000B1
:100B500013F1DAFF6F007BFFF6FF6F0077FFF7FFFF
:100B6000000EF86E0800F550250AD8A4BAEF85F0FB
:100B7000BCEF85F002EF89F060000FF1D9FF600053
:100B800013F1DAFFDE2A000EDD22000E0001636F92
:100B9000000E626F62C066F063C067F064696569E9
:100BA000000ECD6F000ECC6F24EF86F066816000E2
:100BB0000FF1D9FF600013F1DAFFDE2A000EDD220B
:100BC00024EF86F06683D7EF85F06685D7EF85F052
:100BD0006687D7EF85F06689D7EF85F0000ECD6F79
:100BE000010ECC6F24EF86F060000FF1D9FF60009A
:100BF00013F1DAFF6F007BFFF6FF6F0077FFF7FF5F
:100C0000000EF86E0800F550476E486A4850000A1A
:100C1000D8B40DEF86F0EEEF85F04750200AD8B437
:100C2000E8EF85F0030AD8B4EBEF85F0080AD8B4F2
:100C3000E5EF85F0060AD8B4D6EF85F01D0AD8B4E2
:100C4000E2EF85F0EEEF85F0CC51CD11D8B42BEF6B
:100C500086F02DEF86F0F4EF85F066A132EF86F096
:100C600034EF86F035EF86F0669360000FF1D9FF20
:100C7000600013F1DAFF6F007BFFF6FF6F0077FF74
:100C8000F7FF000EF86E0800F5502A0AD8A44BEFC3
:100C900086F04DEF86F080EF86F060000FF1D9FF0F
:100CA000600013F1DAFFDE2A000EDD22600017F18A
:100CB000D9FF60001BF1DAFF6F007CFF47F0020EE6
:100CC000DE266F007CFF48F0000EDD2260001FF181
:100CD000D9FF600023F1DAFF6F0078FF62F06F0048
:100CE00074FF63F063BF79EF86F077EF86F0C2EFB1
:100CF00086F06681626D631FD8B0632BC2EF86F009
:100D000060000FF1D9FF600013F1DAFF6F0078FF88
:100D100009F06F0074FF0AF09BEC90F009C062F0DC
:100D20000AC063F09DEF86F060000FF1D9FF60000C
:100D300013F1DAFFDE2A000EDD22D00E476EFF0E21
:100D4000486E60000FF1D9FF600013F1DAFF6F0009
:100D50007BFFF6FF6F0077FFF7FF000EF86E0800CD
:100D6000F550496E4A6A4750492648504A224A502F
:100D700009E10A0E495CD8A0C0EF86F0C2EF86F008
:100D800094EF86F060000FF1D9FF600013F1DAFFF5
:100D90006F007BFFF6FF6F0077FFF7FF000EF86E26
:100DA0000800F550640AD8B4D8EF86F0DAEF86F080
:100DB000F2EF86F060000FF1D9FF600013F1DAFF67
:100DC0006F007BFFF6FF6F0077FFF7FF000EF86EF6
:100DD0000800F550690AD8A4F0EF86F0F2EF86F02B
:100DE0003DEF87F060000FF1D9FF600013F1DAFFEB
:100DF000DE2A000EDD22600017F1D9FF60001BF132
:100E0000DAFF6F007CFF47F0020EDE266F007CFFEA
:100E100048F0000EDD2260001FF1D9FF600023F1D1
:100E2000DAFF6F0078FFC2F06F0074FFC3F00001BB
:100E3000000EC3BFFF0EC46FC56FC66FC76FC86F0C
:100E4000C96F41C01DF042C01EF0C2C01FF0C3C038
:100E500020F0C4C021F0C5C022F0C6C023F0C7C036
:100E600024F0C8C025F0C9C026F026EC89F01DC0CA
:100E700041F01EC042F025EF89F060000FF1D9FF6C
:100E8000600013F1DAFF6F007BFFF6FF6F0077FF62
:100E9000F7FF000EF86E0800F550730AD8B453EF50
:100EA00087F055EF87F074EF87F060000FF1D9FFFE
:100EB000600013F1DAFF6F0078FF02F06F0074FF3B
:100EC00003F0F70E046EFF0E056E000E076E030EA4
:100ED000066E6BEC94F002500310D8A472EF87F00A
:100EE00074EF87F0CEEF87F060000FF1D9FF60005C
:100EF00013F1DAFF6F007BFFF6FF6F0077FFF7FF5C
:100F0000000EF86E0800F550730AD8B48AEF87F027
:100F10008CEF87F093EF87F0000E0001CF6F030E88
:100F2000CE6F98EF87F0000E0001CF6F010ECE6FED
:100F300060000FF1D9FF600013F1DAFFCE51DE2619
:100F4000CF51DD22600017F1D9FF60001BF1DAFFFD
:100F50006F007CFF47F0020EDE266F007CFF48F03A
:100F6000000EDD2260001FF1D9FF600023F1DAFFDF
:100F70006F0078FFCAF06F0074FFCBF041C00BF038
:100F800042C00CF0CAC00DF0CBC00EF011EC8FF0D7
:100F90000BC041F00CC042F025EF89F060000FF16A
:100FA000D9FF600013F1DAFF6F007BFFF6FF6F00DF
:100FB00077FFF7FF000EF86E0800F550750AD8A409
:100FC000E4EF87F0E6EF87F032EF88F060000FF192
:100FD000D9FF600013F1DAFFDE2A000EDD22600087
:100FE00017F1D9FF60001BF1DAFF6F007CFF47F0BB
:100FF000020EDE266F007CFF48F0000EDD2260004E
:101000001FF1D9FF600023F1DAFF6F0078FF49F08C
:101010006F0074FF4AF049C0D1F04AC0D2F000011D
:10102000D36BD46BD56BD66BD76BD86B41C01DF02F
:1010300042C01EF0D1C01FF0D2C020F0D3C021F0BA
:10104000D4C022F0D5C023F0D6C024F0D7C025F0FC
:10105000D8C026F01CEC8DF01DC041F01EC042F03F
:1010600025EF89F060000FF1D9FF600013F1DAFF7E
:101070006F007BFFF6FF6F0077FFF7FF000EF86E43
:101080000800F550780AD8B448EF88F04AEF88F0A5
:1010900062EF88F060000FF1D9FF600013F1DAFF12
:1010A0006F007BFFF6FF6F0077FFF7FF000EF86E13
:1010B0000800F550580AD8A460EF88F062EF88F075
:1010C000C2EF88F060000FF1D9FF600013F1DAFF82
:1010D0006F007BFFF6FF6F0077FFF7FF000EF86EE3
:1010E00008006F00D4FFD0F060000FF1D9FF60005E
:1010F00013F1DAFFDE2A000EDD22600017F1D9FFBE
:1011000060001BF1DAFF6F007CFF47F0020EDE2665
:101110006F007CFF48F0000EDD2260001FF1D9FF58
:10112000600023F1DAFF6F0078FF49F06F0074FF71
:101130004AF049C0D1F04AC0D2F00001D36BD46B61
:10114000D56BD66BD76BD86B41C01DF042C01EF07B
:10115000D1C01FF0D2C020F0D3C021F0D4C022F003
:10116000D5C023F0D6C024F0D7C025F0D8C026F0D3
:10117000D0C027F099EC8AF01DC041F01EC042F0AB
:1011800025EF89F060000FF1D9FF600013F1DAFF5D
:101190006F007BFFF6FF6F0077FFF7FF000EF86E22
:1011A0000800F550250AD8A4D8EF88F0DAEF88F0C7
:1011B000F3EF88F060000FF1D9FF600013F1DAFF60
:1011C000DE2A000EDD22000E036E250E026E41C0E7
:1011D00004F042C005F06CEC95F0000E426E010E7A
:1011E000416E25EF89F060000FF1D9FF600013F127
:1011F000DAFFDE2A000EDD22000E426E000E416E86
:1012000025EF89F060000FF1D9FF600013F1DAFFDC
:101210006F007BFFF6FF6F0077FFF7FF000EF86EA1
:101220000800F550026E036A41C004F042C005F0A8
:101230006CEC95F060000FF1D9FF600013F1DAFF5C
:10124000DE2A000EDD22EDEF88F012001FC037F01D
:1012500020C038F021C039F022C03AF023C03BF062
:1012600024C03CF025C03DF026C03EF03EBE3BEF22
:1012700089F03EEF89F0010E3FEF89F0000E356EE8
:10128000366A35503610D8B448EF89F04AEF89F005
:101290005AEF89F03E1E3D1E3C1E3B1E3A1E391E73
:1012A000381E376C000E382239223A223B223C226B
:1012B0003D223E22000165BF60EF89F062EF89F0B8
:1012C00063EF89F0669365BF70EF89F0655106E1C1
:1012D0006405D8B06EEF89F070EF89F076EF89F091
:1012E000000E326E010E316E7AEF89F064C031F07B
:1012F00065C032F062C033F063C034F03550361050
:10130000D8A485EF89F087EF89F08EEF89F066A584
:101310008CEF89F08EEF89F091EF89F03306D8A039
:101320003406000E406E1F0E3F6E000E0101966FD8
:1013300016EF8AF03F06D8A04006770E3F24D96EFC
:10134000010E4020DA6E37C002F038C003F039C019
:1013500004F03AC005F03BC006F03CC007F03DC0C9
:1013600008F03EC009F00A0E0A6E000E0B6E000E69
:101370000C6E000E0D6E000E0E6E000E0F6E000E47
:10138000106E000E116E5AEC91F002C027F003C0EF
:1013900028F004C029F005C02AF006C02BF007C0D1
:1013A0002CF008C02DF009C02EF027C014F029C081
:1013B00015F0BDEC9EF01450300FDF6E3106D8A052
:1013C00032063306D8A0340637C002F038C003F026
:1013D00039C004F03AC005F03BC006F03CC007F04D
:1013E0003DC008F03EC009F00A0E0A6E000E0B6EFA
:1013F000000E0C6E000E0D6E000E0E6E000E0F6EC7
:10140000000E106E000E116ED7EC8FF002C037F098
:1014100003C038F004C039F005C03AF006C03BF014
:1014200007C03CF008C03DF009C03EF040BE21EFCF
:101430008AF0405008E13F04D8A021EF8AF023EF62
:101440008AF054EF8AF03750381039103A103B10B8
:101450003C103D103E10D8A430EF8AF032EF8AF0F5
:101460009AEF89F032BE3FEF8AF0325006E1310444
:10147000D8B03DEF8AF03FEF8AF09AEF89F034BEA2
:101480004AEF8AF0345008E13304D8A04AEF8AF0DA
:101490004CEF8AF054EF8AF0000166B352EF8AF005
:1014A00054EF8AF09AEF89F035503610D8A45BEFEC
:1014B0008AF05DEF8AF065EF8AF0000166A563EFC0
:1014C0008AF065EF8AF084EF8AF03F06D8A04006E4
:1014D00035503610D8A46FEF8AF071EF8AF077EFAD
:1014E0008AF0000E306E2B0E2F6E7BEF8AF0000E0E
:1014F000306E2D0E2F6E770E3F24D96E010E4020D8
:10150000DA6E6000BFF0DFFF1DC012F01EC013F0E6
:10151000770E3F24146E010E4020156E33C016F076
:1015200034C017F0A5EC96F012C01DF013C01EF0E9
:101530001200000165BF9FEF8AF0A1EF8AF0A2EFD1
:101540008AF0669365BFAFEF8AF0655106E16405E6
:10155000D8B0ADEF8AF0AFEF8AF0B5EF8AF0000EA9
:10156000316E010E306EB9EF8AF064C030F065C0A4
:1015700031F062C032F063C033F066A9C2EF8AF086
:10158000C4EF8AF0C8EF8AF0FE0E3226FF0E332237
:101590001FC034F020C035F021C036F022C037F033
:1015A00023C038F024C039F025C03AF026C03BF003
:1015B000000E3D6E1F0E3C6E000E0101966F7BEF1C
:1015C0008BF03C06D8A03D060F0E34143E6E3F6AE9
:1015D0003FBEF4EF8AF03F5009E10A0E3E5CD8A00E
:1015E000F4EF8AF0F6EF8AF0FEEF8AF0570E3E2411
:1015F0003E6E000E3F203F6E04EF8BF0300E3E2417
:101600003E6E000E3F203F6EBF0E286EFF0E296E0D
:1016100027502A6E2B6A28502A2629502B222B501D
:1016200007E11A0E2A5CD8B018EF8BF01AEF8BF096
:101630003DEF8BF09F0E286EFF0E296E200E3E10A0
:101640002A6E000E3F102B6E28502A2629502B227E
:101650002B5007E11A0E2A5CD8B031EF8BF033EF34
:101660008BF03DEF8BF03EC008F03FC009F079EC05
:101670009EF008C03EF009C03FF0770E3C24D96EC2
:10168000010E3D20DA6E6000FBF0DFFF3006D8A0CF
:1016900031063206D8A0330634C028F035C029F010
:1016A00036C02AF037C02BF038C02CF039C02DF0EE
:1016B0003AC02EF03BC02FF0050E68EF8BF0D890AB
:1016C0002F322E322D322C322B322A32293228322E
:1016D000E82E5FEF8BF028C034F029C035F02AC027
:1016E00036F02BC037F02CC038F02DC039F02EC0AA
:1016F0003AF02FC03BF03DBE87EF8BF03D5009E143
:10170000020E3C5CD8A087EF8BF089EF8BF0BAEF2C
:101710008BF03450351036103710381039103A101D
:101720003B10D8A496EF8BF098EF8BF0E1EF8AF0A6
:1017300031BEA5EF8BF0315006E13004D8B0A3EFF5
:101740008BF0A5EF8BF0E1EF8AF033BEB0EF8BF0BA
:10175000335008E13204D8A0B0EF8BF0B2EF8BF039
:10176000BAEF8BF0000166B3B8EF8BF0BAEF8BF0F5
:10177000E1EF8AF0000166A9C0EF8BF0C2EF8BF0B9
:10178000D9EF8BF03C06D8A03D06770E3C24D96EED
:10179000010E3D20DA6E60009FF0DFFF3C06D8A00E
:1017A0003D06770E3C24D96E010E3D20DA6E300ED8
:1017B000DF6E1DC012F01EC013F0770E3C24146EB5
:1017C000010E3D20156E32C016F033C017F0A5ECA7
:1017D00096F012C01DF013C01EF01200000E0001A2
:1017E000826F030E836F3D017599738F000E586EE3
:1017F000020E576E57C002F058C003F0E4EC9FF0A1
:101800000009D8B406EF8CF008EF8CF001EF8DF0F2
:1018100058345830536E573000018E6F53C08FF0DC
:1018200082C0D9F083C0DAF03D0EDB6FFC0EDC6FB6
:1018300057C0DDF058C0DEF08EC0DFF08FC0E0F0A2
:10184000E0EC9DF0A7EF8CF082C010F083C011F0A7
:101850005A0E126EFE0E136E3FECA0F0F9EF8CF0F4
:10186000000E026E020E036E850E046EFF0E056EF4
:101870002BEC9CF082C002F083C003F057EC9FF089
:1018800002C055F003C056F0555000018225066E87
:1018900056508321076E000E086E020E096E64EC2E
:1018A0009CF0F9EF8CF082C010F083C011F0620E52
:1018B000126EFF0E136E3FECA0F0F9EF8CF082C0B9
:1018C00010F083C011F03D0E126EFF0E136E3FEC50
:1018D000A0F0F9EF8CF082C010F083C011F0C30EBD
:1018E000126EFF0E136E3FECA0F0F9EF8CF082C089
:1018F00010F083C011F0960E126EFF0E136E3FECC7
:10190000A0F0F9EF8CF082C010F083C011F0DC0E73
:10191000126EFF0E136E3FECA0F0F9EF8CF082C058
:1019200010F083C011F03E0E126EFE0E136E3FECEF
:10193000A0F0F9EF8CF082C010F083C011F0D00E4F
:10194000126EFF0E136E3FECA0F0F9EF8CF08EC01C
:1019500053F08FC054F05450000AD8B4B2EF8CF05A
:101960009BEF8CF05350200AD8B424EF8CF0010A7E
:10197000D8B424EF8CF0030AD8B424EF8CF0010A19
:10198000D8B424EF8CF0040AD8B424EF8CF00F0AFA
:10199000D8B430EF8CF0010AD8B430EF8CF0030AE1
:1019A000D8B430EF8CF01D0AD8B453EF8CF00F0A86
:1019B000D8B45FEF8CF0010AD8B45FEF8CF0030A63
:1019C000D8B45FEF8CF0010AD8B45FEF8CF0070A4F
:1019D000D8B46BEF8CF06B0AD8B477EF8CF03F0A79
:1019E000D8B483EF8CF0C80AD8B48FEF8CF09BEF9B
:1019F0008CF082C002F083C003F0CCEC97F0FDECD9
:101A00009FF0020E5724576E000E5820586E58BE95
:101A100013EF8DF0585009E1FC0E575CD8A013EF7E
:101A20008DF015EF8DF0FAEF8BF03D01739F7599F6
:101A3000738FFDEC9FF01200000165BF22EF8DF067
:101A400024EF8DF025EF8DF0669365BF32EF8DF0BA
:101A5000655106E16405D8B030EF8DF032EF8DF0BE
:101A600038EF8DF0000E306E010E2F6E3CEF8DF0D2
:101A700064C02FF065C030F062C031F063C032F056
:101A80001FC033F020C034F021C035F022C036F042
:101A900023C037F024C038F025C039F026C03AF012
:101AA000000E3C6E1F0E3B6E000E0101966FCFEFD5
:101AB0008DF03B06D8A03C06770E3B24D96E010E74
:101AC0003C20DA6E33C002F034C003F035C004F0BD
:101AD00036C005F037C006F038C007F039C008F04E
:101AE0003AC009F00A0E0A6E000E0B6E000E0C6E64
:101AF000000E0D6E000E0E6E000E0F6E000E106EBC
:101B0000000E116ED8EC95F002C027F003C028F04B
:101B100004C029F005C02AF006C02BF007C02CF045
:101B200008C02DF009C02EF02750300FDF6E2F06B1
:101B3000D8A030063106D8A0320633C002F034C037
:101B400003F035C004F036C005F037C006F038C0E9
:101B500007F039C008F03AC009F00A0E0A6E000E0C
:101B60000B6E000E0C6E000E0D6E000E0E6E000E53
:101B70000F6E000E106E000E116EF4EC94F002C0A9
:101B800033F003C034F004C035F005C036F006C0B1
:101B900037F007C038F008C039F009C03AF03B50C0
:101BA0003C10D8B4D6EF8DF0D8EF8DF009EF8EF061
:101BB00033503410351036103710381039103A10B1
:101BC000D8A4E5EF8DF0E7EF8DF059EF8DF030BE42
:101BD000F4EF8DF0305006E12F04D8B0F2EF8DF025
:101BE000F4EF8DF059EF8DF032BEFFEF8DF03250F3
:101BF00008E13104D8A0FFEF8DF001EF8EF009EF7E
:101C00008EF0000166B307EF8EF009EF8EF059EF0A
:101C10008DF01DC012F01EC013F0770E3B24146E21
:101C2000010E3C20156E31C016F032C017F0A5EC45
:101C300096F012C01DF013C01EF01200000E0F6EC1
:101C4000020E0E6E000E116E000E106E800E000160
:101C50009425D96E020E9521DA6E000EDF6E955135
:101C600007E1160E945DD8B038EF8EF03AEF8EF0A3
:101C700004EF8FF0955109E1130E945DD8A043EF66
:101C80008EF045EF8EF004EF8FF0000E136E020E13
:101C9000126E7DEF8EF0800E1224D96E020E13208C
:101CA000DA6E3B0EDE18D8A458EF8EF05AEF8EF0A5
:101CB0007BEF8EF0800E1224D96E020E1320DA6EA6
:101CC000000EDF6E800E0E24026E020E0F20036ED9
:101CD000D9EC93F02A0E1024D96E010E1120DA6E81
:101CE00060000BF0DFFF104A112A010E12240E6E65
:101CF000000E13200F6E124A132A00019451125C39
:101D000095511358D8A087EF8EF089EF8EF04BEFE6
:101D10008EF0800E0E24026E020E0F20036ED9ECA0
:101D200093F02A0E1024D96E010E1120DA6E600095
:101D30000BF0DFFF2AC1AEF001012B511F0B000198
:101D4000AD6F2CC1ACF02DC1B0F02EC1B1F00101CE
:101D50002F51070B0001AF6FAD51A8ECA0F00001AF
:101D6000AB6F0C0EAB65B7EF8EF0B9EF8EF0BBEF3B
:101D70008EF0000EAB6F070EAF65C1EF8EF0C3EFB4
:101D80008EF0CBEF8EF0000EAF6FFD0E026EFD0EEB
:101D9000036E62EC9DF0000E0001B86F000EB26F92
:101DA000B2C0B9F0B151C8EC9FF00001BA6FB051A8
:101DB000C8EC9FF00001BB6FAFC0BCF0AE51C8ECE7
:101DC0009FF00001BD6FAD51C8EC9FF00001BE6FE8
:101DD000AC51C8EC9FF00001BF6F000EC06FB80E91
:101DE000926F000E936F92C002F093C003F0080E42
:101DF000046E680ECEEC9CF08C0E026EFE0E036E2E
:101E000062EC9DF010EF8FF0A30E026EFB0E036EDE
:101E100062EC9DF02D0E026EFB0E036E62EC9DF0E7
:101E2000120020EED9F110EE10F0060E6F006FFFD9
:101E3000E3FFE806FBE20DC01BF00EC01CF01B50D8
:101E40001C10D8A426EF8FF028EF8FF02CEF8FF026
:101E5000100E1B6E000E1C6E1BC002F01CC003F0A7
:101E600057EC9FF002C01FF003C020F064C01DF0CB
:101E700065C01EF01EBE3FEF8FF041EF8FF056EFB2
:101E80008FF01F501D5C1E50800A0F6E2050800A7C
:101E90000F58D8A04EEF8FF050EF8FF052EF8FF029
:101EA00056EF8FF01DC01FF01EC020F01FC01DF0A8
:101EB00020C01EF062C019F063C01AF0000166B1C4
:101EC00064EF8FF066EF8FF083EF8FF074EF8FF099
:101ED000000E036E200E026E0BC004F00CC005F065
:101EE0006CEC95F01F4A202A19501F5C2050800A84
:101EF0000F6E1A50800A0F58D8A081EF8FF083EF31
:101F00008FF068EF8FF0000E186E000E176E9EEFC8
:101F10008FF060006FF0D9FF600073F0DAFFDF50E0
:101F20000F6E0F50026E036A0BC004F00CC005F078
:101F30006CEC95F01B4A1C2A174A182A1D50175C96
:101F40001850800A0F6E1E50800A0F58D8A0ABEFB1
:101F50008FF0ADEF8FF089EF8FF0000166A1B3EF46
:101F60008FF0B5EF8FF0D2EF8FF0C3EF8FF0000E50
:101F7000036E200E026E0BC004F00CC005F06CEC7A
:101F800095F01F4A202A19501F5C2050800A0F6EBE
:101F90001A50800A0F58D8A0D0EF8FF0D2EF8FF0F0
:101FA000B7EF8FF01FC00BF020C00CF01200000E36
:101FB000136E11BEE0EF8FF0DEEF8FF0F2EF8FF0D7
:101FC000111E101E0F1E0E1E0D1E0C1E0B1E0A6C67
:101FD000000E0B220C220D220E220F2210221122A3
:101FE000010E136E09BEF9EF8FF0F7EF8FF00BEFD4
:101FF00090F0091E081E071E061E051E041E031E65
:10200000026C000E03220422052206220722082267
:102010000922010E131A20EE14F0070EDE6AE806FC
:10202000FDE20A500B100C100D100E100F101010C6
:102030001110D8B41EEF90F020EF90F072EF90F0F6
:10204000010E126E2EEF90F0D8900A360B360C3639
:102050000D360E360F3610361136122A11AE33EF0A
:1020600090F035EF90F024EF90F0D89014361536BC
:1020700016361736183619361A361B360A50025CD1
:102080000B5003580C5004580D5005580E5006586C
:102090000F5007581050085811500958D8A053EF46
:1020A00090F055EF90F066EF90F00A50025E0B5002
:1020B000035A0C50045A0D50055A0E50065A0F5030
:1020C000075A1050085A1150095A1480D8901132EA
:1020D00010320F320E320D320C320B320A32122E07
:1020E00035EF90F01350D8B478EF90F07AEF90F08D
:1020F0008AEF90F01B1E1A1E191E181E171E161EA0
:10210000151E146C000E15221622172218221922F1
:102110001A221B2214C002F015C003F016C004F0EE
:1021200017C005F018C006F019C007F01AC008F073
:102130001BC009F01200000E126E000E116E000E90
:10214000106E000E0F6EA7EF90F0094A0A2A600089
:1021500027F0F6FF60002BF0F7FF000EF86E080086
:10216000F550200AD8B4B7EF90F0B9EF90F0A5EF92
:1021700090F0F70E0B6EFF0E0C6E600027F0F6FF6E
:1021800060002BF0F7FF000EF86E0800F5500D6EA2
:102190000E6A0B500D260C500E220E5009E1050E52
:1021A0000D5CD8A0D6EF90F0D8EF90F0A5EF90F0AE
:1021B000E2EF90F0000E106E010E0F6E094A0A2A2F
:1021C0001FEF91F0600027F0F6FF60002BF0F7FFA3
:1021D000000EF86E0800F5500B6E0C6A0C50000AE9
:1021E000D8B4F5EF90F01FEF91F00B502B0AD8B454
:1021F000DEEF90F0060AD8B4DAEF90F01FEF91F01E
:1022000011C002F012C003F0000E056E0A0E046E3B
:102210002AECA0F0600027F0F6FF60002BF0F7FF3B
:10222000000EF86E0800F550025E000E035A300EE4
:102230000224116E000E0320126EDEEF90F0D00E1D
:102240000B6EFF0E0C6E600027F0F6FF60002BF0A7
:10225000F7FF000EF86E0800F5500D6E0E6A0B5079
:102260000D260C500E220E5009E10A0E0D5CD8A06E
:102270003CEF91F03EEF91F000EF91F00F50101015
:10228000D8A445EF91F047EF91F055EF91F011C0D0
:102290000BF012C00CF00B1E0C1E0B4A0C2A0BC0CC
:1022A00009F00CC00AF059EF91F011C009F012C00A
:1022B0000AF01200000E136E09BE63EF91F061EF99
:1022C00091F075EF91F0091E081E071E061E051EEF
:1022D000041E031E026C000E0322042205220622A5
:1022E000072208220922010E136E11BE7CEF91F025
:1022F0007AEF91F08CEF91F0111E101E0F1E0E1E42
:102300000D1E0C1E0B1E0A6C000E0B220C220D2241
:102310000E220F22102211220A500B100C100D1049
:102320000E100F1010101110D8B499EF91F09BEF10
:1023300091F0E3EF91F0010E126EA9EF91F0D890B9
:102340000A360B360C360D360E360F361036113671
:10235000122A11AEAEEF91F0B0EF91F09FEF91F035
:102360000A50025C0B5003580C5004580D5005588D
:102370000E5006580F500758105008581150095861
:10238000D8A0C5EF91F0C7EF91F0D7EF91F00A50C8
:10239000025E0B50035A0C50045A0D50055A0E5051
:1023A000065A0F50075A1050085A1150095AD8901F
:1023B000113210320F320E320D320C320B320A3221
:1023C000122EB0EF91F01350D8B4E9EF91F0EBEF8B
:1023D00091F0FBEF91F0091E081E071E061E051E58
:1023E000041E031E026C000E032204220522062294
:1023F00007220822092202C002F003C003F004C031
:1024000004F005C005F006C006F007C007F008C0DC
:1024100008F009C009F01200400E25EC9AF0030EF6
:102420000B6E080E0A6E770EE82EFED70A2EFCD72A
:102430000B2EFAD700F0000E0D6E000E0C6E080485
:102440000910D8A426EF92F028EF92F030EF92F026
:10245000850E026EF70E036E62EC9DF0FDEC9FF0B0
:10246000000E0F6E000E0E6E08040910D8A43BEF8C
:1024700092F03DEF92F06EEF92F00E500F10D8B444
:1024800044EF92F046EF92F06EEF92F0070E0E14CA
:102490000A6E000E0F140B6E0A500B10D8A453EFE7
:1024A00092F055EF92F06EEF92F00CC00AF00DC072
:1024B0000BF0D8900A360B36D8900A360B36D890E7
:1024C0000A360B36850E0A24026EF70E0B20036EB9
:1024D00062EC9DF00C4A0D2AFDEC9FF05D0E0E247F
:1024E000F66EF60E0F20F76EF86A000EF82208005E
:1024F000F550F1EC9BF008040910D8A482EF92F09B
:1025000084EF92F093EF92F05D0E0E24F66EF60ECD
:102510000F20F76EF86A000EF8220800F55056EC0E
:102520009EF0FDEC9FF00E4A0F2A0F5009E1400E7D
:102530000E5CD8A09EEF92F0A0EF92F034EF92F0F4
:10254000800E25EC9AF0D00E0A6ECA0EE82EFED749
:102550000A2EFCD71200FB0E026EFF0E036E62EC19
:102560009DF0000E046E300E3BEC9BF0680E086E82
:10257000E40EE82EFED7082EFCD700D0320E63EC16
:10258000A0F0000E046E300E3BEC9BF0150E086EB2
:10259000C60EE82EFED7082EFCD700D0330E63EC13
:1025A000A0F0000E046E300E3BEC9BF0150E086E92
:1025B000C60EE82EFED7082EFCD700D0340E63ECF2
:1025C000A0F0000E046E250E3BEC9BF0150E086E7D
:1025D000C60EE82EFED7082EFCD700D0350E63ECD1
:1025E000A0F0010E046E280E3BEC9BF0150E086E59
:1025F000C60EE82EFED7082EFCD700D0360E63ECB0
:10260000A0F0010E046E080E3BEC9BF0150E086E58
:10261000C60EE82EFED7082EFCD700D0370E63EC8E
:10262000A0F0010E046E010E3BEC9BF0030E096E50
:10263000080E086E770EE82EFED7082EFCD7092E5E
:10264000FAD700F0380E63ECA0F0010E046E060E0F
:102650003BEC9BF0150E086EC60EE82EFED7082E3A
:10266000FCD700D0390E63ECA0F0010E046E0C0E06
:102670003BEC9BF0150E086EC60EE82EFED7082E1A
:10268000FCD700D0410E63ECA0F01200096ED9EC2B
:1026900099F0000E0001F66F000E0101E06FF60EDA
:1026A000026E000E036E0001B05139EC9FF0480E2F
:1026B0000001F86FF90E026E000E036EB15139EC95
:1026C0009FF04D0E0001FB6FFC0E026E000E036EBC
:1026D000B25139EC9FF0530E0001FE6F000EFF6FF8
:1026E000E00E026E010E036EAE5139EC9FF02F0E1C
:1026F0000101E26FE30E026E010E036E0001AD51A7
:1027000039EC9FF02F0E0101E56FE60E026E010E0F
:10271000036E0001AC5139EC9FF0000E0101E86F2F
:102720000001AD51A8ECA0F00001AB6FB051A8ECD6
:10273000A0F00001AA6FB151A8ECA0F00001A86FB1
:10274000B251A8ECA0F00001A96F0904D8A4ABEF26
:1027500093F0ADEF93F0D8EF93F0AF51020DC90EA7
:10276000F324D96E010EF420DA6E6F0078FF02F0C8
:102770006F0074FF03F0CCEC97F0200E63ECA0F038
:10278000E00E026E010E036ECCEC97F0E80E026EC6
:10279000F90E036E62EC9DF0F60E026E000E036EF3
:1027A000CCEC97F0E80E026EF90E036E62EC9DF031
:1027B0001200DDEF93F0024A032A60000BF0D9FF0C
:1027C00060000FF0DAFF200EDE18D8B4EAEF93F0C5
:1027D000ECEF93F0DBEF93F060000BF0D9FF6000BB
:1027E0000FF0DAFF090EDE18D8B4F9EF93F0FBEF23
:1027F00093F0DBEF93F0000E076E000E066E6000A4
:102800000BF0D9FF60000FF0DAFF2D0EDE18D8A410
:102810000CEF94F00EEF94F013EF94F0062A024AB6
:10282000032A36EF94F060000BF0D9FF60000FF040
:10283000DAFF2B0EDE18D8A420EF94F022EF94F0EC
:1028400036EF94F0024A032A36EF94F060000BF062
:10285000D9FF60000FF0DAFFDF50046E07500A0D59
:10286000F3500424D00F076E22EF94F060000BF0B9
:10287000D9FF60000FF0DAFF2F0EDF6442EF94F013
:1028800044EF94F052EF94F060000BF0D9FF600039
:102890000FF0DAFF390EDF6450EF94F052EF94F04E
:1028A00026EF94F00650D8B458EF94F05AEF94F015
:1028B00067EF94F00750046E056A041E051E044A73
:1028C000052A04C002F005C003F06AEF94F007C0C7
:1028D00002F0036A120002C009F003C00AF004C04B
:1028E0000BF005C00CF00606D8A00706062806E186
:1028F0000728D8A47EEF94F080EF94F08DEF94F049
:10290000000E036E000E026EF3EF94F0094A0A2ADD
:102910000B4A0C2A0606D8A00706600027F0F6FF2F
:1029200060002BF0F7FF000EF86E0800F55000096C
:10293000D8B49DEF94F09FEF94F0D8EF94F060003E
:102940002FF0F6FF600033F0F7FF000EF86E08007E
:10295000F5500009D8B4AFEF94F0B1EF94F0D8EF90
:1029600094F006500710D8B4B8EF94F0BAEF94F092
:10297000D8EF94F0600027F0F6FF60002BF0F7FF2F
:10298000000EF86E08006F00D4FF08F060002FF012
:10299000F6FF600033F0F7FF000EF86E0800F55008
:1029A0000818D8B4D6EF94F0D8EF94F086EF94F0EE
:1029B000600027F0F6FF60002BF0F7FF000EF86EC6
:1029C00008006F00D4FF08F060002FF0F6FF6000F1
:1029D00033F0F7FF000EF86E0800F550085C026E49
:1029E000036AD8A00306120020EE12F0070EDE6A7A
:1029F000E806FDE20A500B100C100D100E100F101F
:102A000010101110D8B407EF95F009EF95F05BEFB7
:102A100095F0010E1A6E17EF95F0D8900A360B3626
:102A20000C360D360E360F36103611361A2A11AE08
:102A30001CEF95F01EEF95F00DEF95F0D890123643
:102A400013361436153616361736183619360A5018
:102A5000025C0B5003580C5004580D5005580E5092
:102A600006580F5007581050085811500958D8A050
:102A70003CEF95F03EEF95F04FEF95F00A50025E77
:102A80000B50035A0C50045A0D50055A0E50065A5A
:102A90000F50075A1050085A1150095A1280D890F6
:102AA000113210320F320E320D320C320B320A322A
:102AB0001A2E1EEF95F012C002F013C003F014C0DE
:102AC00004F015C005F016C006F017C007F018C0D6
:102AD00008F019C009F0120004500510D8B473EFC3
:102AE00095F075EF95F07EEF95F004500510D8A4A1
:102AF0007CEF95F07EEF95F083EF95F00250B9EC06
:102B0000A0F0D7EF95F020EE09F00450D92605503B
:102B1000DA22DE50DE10D8B490EF95F092EF95F007
:102B2000ADEF95F020EE09F00450D9260550DA22D9
:102B300010EE03F00450E1260550E222DE50E65C80
:102B4000E650800A0A6EDE50800A0A58D8B0ABEF11
:102B500095F0ADEF95F0D7EF95F020EE03F004502F
:102B6000D9260550DA226F0078FF06F06F0074FF57
:102B700007F0600013F0D9FF600017F0DAFF6F0074
:102B800078FF08F06F0074FF09F006500824D96E32
:102B900007500920DA6E60000BF0DFFF20EE03F033
:102BA0000450D9260550DA22DE2A000EDD2212005A
:102BB0000A500B100C100D100E100F1010101110E9
:102BC000D8B4E5EF95F0E7EF95F02FEF96F0010E12
:102BD000126EF5EF95F0D8900A360B360C360D369E
:102BE0000E360F3610361136122A11AEFAEF95F066
:102BF000FCEF95F0EBEF95F00A50025C0B50035898
:102C00000C5004580D5005580E5006580F500758D8
:102C10001050085811500958D8A011EF96F013EF32
:102C200096F023EF96F00A50025E0B50035A0C50B8
:102C3000045A0D50055A0E50065A0F50075A10509C
:102C4000085A1150095AD890113210320F320E32F0
:102C50000D320C320B320A32122EFCEF95F002C00C
:102C600002F003C003F004C004F005C005F006C084
:102C700006F007C007F008C008F009C009F012000C
:102C80007AEF96F0800E25EC9AF0240E066EF90E7F
:102C9000076EB5EC9AF0800E25EC9AF098EF96F05E
:102CA000C00E25EC9AF0240E066EF90E076EB5ECF8
:102CB0009AF0C00E25EC9AF098EF96F0940E25EC61
:102CC0009AF0240E066EF90E076EB5EC9AF0940E8B
:102CD00025EC9AF098EF96F0D40E25EC9AF0240E9D
:102CE000066EF90E076EB5EC9AF0D40E25EC9AF04C
:102CF00098EF96F00CC00EF00DC00FF00F50000AC8
:102D0000D8B485EF96F098EF96F00E50010AD8B43B
:102D100042EF96F0030AD8B450EF96F0010AD8B407
:102D20005EEF96F0070AD8B46CEF96F098EF96F045
:102D3000090E0F6E1E0E0E6EE40EE82EFED70E2E3E
:102D4000FCD70F2EFAD700D01200000166A1ABEF1E
:102D500096F0ADEF96F0B7EF96F014C00BF015C0FB
:102D60000CF012C00DF013C00EF09BEC9EF017BEDD
:102D7000BCEF96F0BEEF96F0C4EF96F016C01BF0D5
:102D800017C01CF0C8EF96F0000E1C6E000E1B6EF4
:102D9000000E1A6E000E196EDAEF96F0000E036E3A
:102DA000200E026E12C004F013C005F06CEC95F01A
:102DB000194A1A2A1B50195C1A50800A186E1C50A6
:102DC000800A1858D8A0E7EF96F0E9EF96F0CEEF1A
:102DD00096F0000166B1EFEF96F0F1EF96F0FBEFA1
:102DE00096F014C00BF015C00CF012C00DF013C01B
:102DF0000EF09BEC9EF014C002F015C003F057ECEF
:102E00009FF01B500224126E1C500320136E120000
:102E1000000E076E05BE11EF97F00FEF97F017EF5A
:102E200097F0046C051ED8B0052A010E076E03BE8C
:102E30001EEF97F01CEF97F024EF97F0026C031E43
:102E4000D8B0032A010E071A000E096E000E086E94
:102E500004500510D8B42FEF97F031EF97F059EFE9
:102E600097F0010E066E39EF97F0D89004360536CC
:102E7000062A05AE3EEF97F040EF97F035EF97F05A
:102E8000D890083609360450025C05500358D8A083
:102E90004CEF97F04EEF97F053EF97F00450025E2F
:102EA0000550035A0880D89005320432062E40EFB0
:102EB00097F00750D8B45FEF97F061EF97F065EFA8
:102EC00097F0086C091ED8B0092A08C002F009C0A2
:102ED00003F012000A500001F45DF551800A0D6EF6
:102EE0000B50800A0D58D8B078EF97F07AEF97F032
:102EF0007EEF97F0F4C00AF0F5C00BF0080409105B
:102F0000D8A485EF97F087EF97F08BEF97F00A50F2
:102F10007F0F25EC9AF0020E08180910D8A493EF41
:102F200097F095EF97F099EF97F00A50BF0F25ECC7
:102F30009AF0030E08180910D8A4A1EF97F0A3EF98
:102F400097F0A7EF97F00A50930F25EC9AF0040E34
:102F500008180910D8A4AFEF97F0B1EF97F0B5EFCC
:102F600097F00A50D30F25EC9AF0030E0E6E080E60
:102F70000D6E770EE82EFED70D2EFCD70E2EFAD74B
:102F800000F00C50F1EC9BF0D00E0D6ECA0EE82E46
:102F9000FED70D2EFCD71200000E076E000E066E37
:102FA00009EF98F03901A3A9D8EF97F0DAEF97F07D
:102FB000D2EF97F006500224046E07500320056EEE
:102FC000600013F0F6FF600017F0F7FF000EF86ED8
:102FD0001F0EF76403D00800F55007D06F00DBFF29
:102FE000E9FF6F00DFFFEAFFEF503D01EA6F064A9D
:102FF000072A07BE05EF98F0075009E1810E065C2D
:10300000D8A005EF98F007EF98F009EF98F02CEFB3
:1030100098F006500224046E07500320056E6000ED
:1030200013F0F6FF600017F0F7FF000EF86E1F0EAA
:10303000F76403D00800F55007D06F00DBFFE9FF0D
:103040006F00DFFFEAFFEF500009D8A42AEF98F0E5
:103050002CEF98F0D2EF97F01200000EBA6EBB681A
:10306000000EBC6E030EC26EC368A70EC46E000EC7
:103070003A01606F000E506F000E406F000E816FBE
:103080005169FC0E416FC00E616F000E006F000EA3
:10309000016F000E026F000E036F000E086F000E2E
:1030A000096F000E0A6F000E0B6F000E0C6F000E02
:1030B0000D6F000E0E6F000E0F6F070E426F000EA9
:1030C000526F180E626F43695369636944695469AA
:1030D0006469080E846F000E476F000E466F000E85
:1030E000456F000E576F7F0E566F000E556F000E26
:1030F000676F000E666F000E656F000E156F210E74
:10310000136F220E146F130E166F170EE56F130E4A
:10311000E16F140EE26F12000C6E0850D8A493EF0A
:1031200098F095EF98F097EF98F0010E086E085020
:10313000096E0A6A09500001F45DF551800A0B6EB0
:103140000A50800A0B58D8B0A8EF98F0AAEF98F070
:10315000ACEF98F0F405086E0C04D8A4B2EF98F028
:10316000B4EF98F0B8EF98F008507F0F25EC9AF084
:10317000020E0C18D8A4BFEF98F0C1EF98F0C5EF7D
:1031800098F00850BF0F25EC9AF0030E0C18D8A445
:10319000CCEF98F0CEEF98F0D2EF98F00850930F64
:1031A00025EC9AF0040E0C18D8A4D9EF98F0DBEFB8
:1031B00098F0DFEF98F00850D30F25EC9AF0D00E7E
:1031C000096ECA0EE82EFED7092EFCD71200000E9B
:1031D000076E03BEF0EF98F0EEEF98F0F6EF98F080
:1031E000026C031ED8B0032A010E076E05BEFDEF68
:1031F00098F0FBEF98F001EF99F0046C051ED8B041
:10320000052A04500510D8B408EF99F00AEF99F098
:103210002EEF99F0010E066E12EF99F0D890043659
:103220000536062A05AE17EF99F019EF99F00EEF63
:1032300099F00450025C05500358D8A022EF99F091
:1032400024EF99F028EF99F00450025E0550035ADC
:10325000D89005320432062E19EF99F00750D8B4F1
:1032600034EF99F036EF99F03AEF99F0026C031EC3
:0E327000D8B0032A02C002F003C003F012001F
:103280003901A3A746EF99F048EF99F08CEF99F038
:1032900093A74DEF99F04FEF99F08CEF99F06F00F5
:1032A000A0F7B5F00D0E0001B519D8B45AEF99F09A
:1032B0005CEF99F067EF99F0855109E1800E845D2C
:1032C000D8A065EF99F067EF99F07DEF99F0010EC6
:1032D000B66F800E8425D96E020E8521DA6E000E3F
:1032E000DF6E84C094F085C095F0000E856F000EEF
:1032F000846F390193978CEF99F0800E8425D96EF5
:10330000020E8521DA6E6000D7F2DFFF844B852B39
:1033100084C094F085C095F011006E0EF66E3B0EE1
:10332000F76E010EF86E00EE97F110EE52F0090004
:103330006F00D7FFEEFFE550E150F9E1660EF66E43
:10334000410EF76E010EF86E00EEF4F010EE0CF088
:1033500009006F00D7FFEEFFE550E150F9E100EE04
:1033600000F3800EEE6AE806FDE100EE00F210EEDA
:1033700000F1EE6AE550E150FCE1E250FAE100EEC6
:1033800000F1970EEE6AE806FDE100EE60F0620ED5
:10339000EE6AE806FDE15D6A5C6A5B6A5A6A596A30
:1033A000080ED56E000ED66E000ED76E000100EF2F
:1033B00080F0000E086E000E076EB80E0724D96E5E
:1033C000000E0820DA6E000EDF6E074A082A08BEDB
:1033D000F3EF99F0085009E1090E075CD8A0F3EF6C
:1033E00099F0F5EF99F0DDEF99F0B80E0001926FCA
:1033F000000E936F000E026E92C003F093C004F0B3
:10340000070E056E680E79EC9BF0B8C0B2F0B9C03B
:10341000B1F00001BA513F0BB06FBBC0AFF0070E67
:10342000AF6515EF9AF017EF9AF019EF9AF0000ECA
:10343000AF6FBCC0AEF0BD511F0BAD6FBEC0ACF0E6
:10344000000EBF6F000EC06F1200066E0650F00B2C
:103450000C09076E07C002F05D501BEC9FF014ECE6
:10346000A0F00650F00B0809076E07C002F05D508F
:103470001BEC9FF014ECA0F006C004F00F0E041635
:103480000438F00B0C09076E07C002F05D501BEC0E
:103490009FF014ECA0F006C004F00F0E04160438E0
:1034A000F00B0809076E07C002F05D501BEC9FF09F
:1034B00014ECA0F00604D8A460EF9AF062EF9AF042
:1034C0006EEF9AF0090E056E1E0E046EE40EE82EE5
:1034D000FED7042EFCD7052EFAD700D01200076EB7
:1034E0003D0177AF76EF9AF078EF9AF070EF9AF0AF
:1034F000075007246E6F020E6C6F03506B6F799547
:10350000738B78AB86EF9AF088EF9AF081EF9AF0A0
:1035100060000BF06BFD79A590EF9AF092EF9AF0B6
:103520008BEF9AF06E2B60001BF06CFD738BABEF92
:103530009AF078A19EEF9AF0A0EF9AF099EF9AF0A6
:10354000600013F0D9FF600017F0DAFF6F00ABF5F1
:10355000DFFF044A052A06060628D8A4B2EF9AF02F
:10356000B4EF9AF099EF9AF01200000E0B6E000E75
:103570000A6ED1EF9AF00A500624086E0B5007200D
:10358000096E600023F0F6FF600027F0F7FF000EE1
:10359000F86E0800F550F1EC9BF00A4A0B2A14EC87
:1035A000A0F00A500624086E0B500720096E600038
:1035B00023F0F6FF600027F0F7FF000EF86E08001A
:1035C000F5500009D8B4E7EF9AF0E9EF9AF0F9EF77
:1035D0009AF00001F4510A5C0B50800A086EF55114
:1035E000800A0858D8A0F7EF9AF0F9EF9AF0BBEFED
:1035F0009AF01200076E3D0177AF01EF9BF003EFE9
:103600009BF0FBEF9AF0075007246E6F0650020FF5
:103610006C6F03506B6F738B78AB11EF9BF013EFF4
:103620009BF00CEF9BF060000BF06BFD79A51BEF9E
:103630009BF01DEF9BF016EF9BF0738B31EF9BF02F
:1036400078AB25EF9BF027EF9BF020EF9BF060001D
:1036500013F0D9FF600017F0DAFFDF506B6F044AF8
:10366000052A06060628D8A438EF9BF03AEF9BF00F
:1036700020EF9BF01200066E0650F00B0C09076E4F
:1036800007C002F05D501BEC9FF014ECA0F0065058
:10369000F00B0809076E07C002F05D501BEC9FF0AD
:1036A00014ECA0F00404D8A458EF9BF05AEF9BF060
:1036B00078EF9BF006C005F00F0E05160538F00BED
:1036C0000C09076E07C002F05D501BEC9FF014EC74
:1036D000A0F006C005F00F0E05160538F00B08091E
:1036E000076E07C002F05D501BEC9FF014ECA0F0D9
:1036F0001200066E065006243D016E6F60000BF04E
:103700006BFD010E6C6F738D738B73A78AEF9BF04B
:103710008CEF9BF085EF9BF006500624066E06505A
:1037200001096E6F600017F06CFD738B739DABEF3A
:103730009BF078A19EEF9BF0A0EF9BF099EF9BF0A0
:1037400060000FF0D9FF600013F0DAFF6F00ABF5F7
:10375000DFFF034A042A6C51D8A4B1EF9BF0B3EF0A
:103760009BF099EF9BF09CECA0F012003901A3A70D
:10377000BCEF9BF0BEEF9BF0C1EF9BF06F00A0F79A
:10378000B5F0000E036E000E026E800E0224D96E9C
:10379000020E0320DA6E000EDF6E024A032A035087
:1037A00009E17F0E025CD8A0D8EF9BF0DAEF9BF026
:1037B000C5EF9BF0000E0001B66F3D01F289000ECF
:1037C000F96F000EFA6F000E0201806F000E00010B
:1037D000956F000E946F000EB56F3901938D93872E
:1037E0001200056E0550F00B0D090001B76FB7C050
:1037F00002F05D501BEC9FF014ECA0F00550F00BB4
:1038000009090001B76FB7C002F05D501BEC9FF0D3
:1038100014ECA0F005C004F00F0E04160438F00BF1
:103820000D090001B76FB7C002F05D501BEC9FF0AF
:1038300014ECA0F005C004F00F0E04160438F00BD1
:1038400009090001B76FB7C002F05D501BEC9FF093
:1038500014ECA0F01200600013F0F6FF600017F007
:10386000F7FF000EF86E08006F00D4FFB4F052EFBF
:103870009CF0600013F0F6FF600017F0F7FF000EF9
:10388000F86E08006F00D4FFB4F060000BF0D9FFB1
:1038900060000FF0DAFF6000D3F2DFFF024A032A74
:1038A000044A052A0001B451D8A459EF9CF05BEFFB
:1038B0009CF039EF9CF060000BF0D9FF60000FF036
:1038C000DAFF000EDF6E120008C00CF009C00DF028
:1038D00006C00EF007C00FF00C500A6E0D500B6EB4
:1038E0000C4A0D2A60002BF0F6FF60002FF0F7FF66
:1038F000000EF86E60003BF0D9FF60003FF0DAFF89
:103900000E4A0F2A1F0EF76403D00800F55007D0A7
:103910006F00DBFFE9FF6F00DFFFEAFFEF50DF6EB4
:10392000DF50D8A496EF9CF098EF9CF06CEF9CF0E1
:1039300012004DC051F04EC052F0000E0001616FF8
:10394000000E606FB7EF9CF04BC041F04CC042F0EE
:10395000510E436E000E446E4FC045F050C046F00D
:10396000A4EC85F0415000016027425061236000C3
:1039700047F1F6FF60004BF1F7FF000EF86E08000C
:10398000F5500009D8A4C7EF9CF0C9EF9CF0A4EF54
:103990009CF060C04BF061C04CF01200056E02C09C
:1039A00006F003C007F0055005243D016E6F60006E
:1039B0001BF0D9FF60001FF0DAFFDF506B6F600073
:1039C00013F06CFD738BF6EF9CF078ABEAEF9CF094
:1039D000ECEF9CF0E5EF9CF060001BF0D9FF60007D
:1039E0001FF0DAFFDF506B6F064A072A6C51D8A42C
:1039F000FCEF9CF0FEEF9CF0E5EF9CF09CECA0F05F
:103A00001200000E0A6E000E096E14EF9DF00950B0
:103A10000624D96E0A500720DA6EDF50F1EC9BF0D5
:103A200014ECA0F0094A0A2A09500624D96E0A505B
:103A30000720DA6EDF50D8B420EF9DF022EF9DF022
:103A400032EF9DF00001F451095C0A50800A086EC3
:103A5000F551800A0858D8A030EF9DF032EF9DF064
:103A600007EF9DF01200066E03C007F004C008F0D7
:103A7000065006243D016E6F60000BF06BFD052AB9
:103A8000600017F06CFD738B57EF9DF078AB4BEF38
:103A90009DF04DEF9DF046EF9DF060001FF0D9FFC7
:103AA000600023F0DAFFDF506B6F074A082A6C5181
:103AB000D8A45DEF9DF05FEF9DF046EF9DF09CEC8C
:103AC000A0F012007AEF9DF03901A3A96AEF9DF0F2
:103AD0006CEF9DF064EF9DF060000BF0F6FF60006E
:103AE0000FF0F7FF000EF86E08006F00D7FFEAFD39
:103AF000024A032A60000BF0F6FF60000FF0F7FFA8
:103B0000000EF86E0800F5500009D8A48AEF9DF069
:103B10008CEF9DF064EF9DF01200056E000E000129
:103B2000696F000E686FA4EF9DF0520E036E2B0EAE
:103B3000026E000EE82EFED7022EFCD7032EFAD717
:103B400000D00001684B692B0550026E036A0250D9
:103B5000685D6951800A046E0350800A0458D8A039
:103B6000B4EF9DF0B6EF9DF095EF9DF01200A2F935
:103B700091F988F9D9F9C6F9DFF9D3F97FF9CDF9C7
:103B800039F976F96CF962F934F844F764F8DFF83A
:103B900005F9B4F6FEF702F790F8B9F8E4F9C5F7BD
:103BA000BFF9B8F9B1F958F9AAF94EF99AF944F9F7
:103BB000286E756C6C290030302F30302F3030007B
:103BC000DD0E0001E76F000EE86FD9C0E9F0DAC042
:103BD000EAF0000EED6F000EEC6F000EF36F000EBA
:103BE000F26FE90E4B6E000E4C6EDBC04DF0DCC088
:103BF0004EF0E70E4F6E000E506E99EC9CF00001F7
:103C0000EC51D925D96EED51DA21DA6E000EDF6E56
:103C10001200010E086E200E02180310D8B413EF24
:103C20009EF015EF9EF02EEF9EF0F70E046EFF0E45
:103C3000056E02C006F003C007F0045006260550CA
:103C40000722075009E1050E065CD8A02AEF9EF076
:103C50002CEF9EF02EEF9EF0000E086E08C002F0D2
:103C6000036A1200000E3D01EC6F000EED6F000EB6
:103C7000EE6F000EEF6F000EF06F000EF16FB00EE2
:103C8000F26F800EF36F000EF46F8A0EF56F000E68
:103C9000F66F000EF76F000EF86F000EF96F000E52
:103CA000FA6FF28BF289390193971200036E800E3E
:103CB000046E70EF9EF0035004140009D8B463EF53
:103CC0009EF065EF9EF06AEF9EF02A0E63ECA0F086
:103CD0006DEF9EF0200E63ECA0F0D8900430046EDF
:103CE0000450D8A476EF9EF078EF9EF05BEF9EF044
:103CF00012009F0E0A6EFF0E0B6E08C00CF009C07A
:103D00000DF00A500C260B500D220D5007E11A0E33
:103D10000C5CD8B08EEF9EF090EF9EF096EF9EF088
:103D20005F0E0814086E096A9AEF9EF008C008F04A
:103D300009C009F01200000E116E000E106EACEFFB
:103D40009EF00FC002F0036A0DC004F00EC005F033
:103D50006CEC95F0104A112A10500B24D96E1150BA
:103D60000C20DA6EDF500F6E0F50D8A4BAEF9EF021
:103D7000BCEF9EF0A1EF9EF0120015BECAEF9EF0C0
:103D8000155006E11404D8B0C8EF9EF0CAEF9EF0BB
:103D9000D8EF9EF014C016F015C017F0161E171EAF
:103DA000164A172A16C014F017C015F0DCEF9EF063
:103DB00014C014F015C015F01200D28AD250D29E51
:103DC000D29CD28A550ED46EAA0ED46ED490000E18
:103DD000D76E000ED66E080ED56E550ED46EAA0E96
:103DE000D46ED4803901838781818491839F8495A7
:103DF00087918991809FD29E12009F0E046EFF0EC4
:103E0000056E200E0210066E000E0310076E0450A1
:103E100006260550072207500AE11A0E065CD8A0B4
:103E200014EF9FF017EF9FF0010E18EF9FF0000EB8
:103E3000026E036A1200036E3D0177AF22EF9FF01E
:103E400024EF9FF01CEF9FF0035003246E6F010ED0
:103E50006C6F60000BF06BFD738B78AB32EF9FF0F3
:103E600034EF9FF02DEF9FF0350EE82EFED700F0D7
:103E70001200046E04380F0B300F60000BF0D9FFF6
:103E800060000FF0DAFFDF6E20EE01F00250D9265D
:103E90000350DA2204500F0B300FDF6E20EE02F0D9
:103EA0000250D9260350DA22000EDF6E120002C043
:103EB00004F003C005F05FEF9FF0024A032A6000A0
:103EC0000BF0D9FF60000FF0DAFFDF50D8A46BEFE2
:103ED0009FF06DEF9FF05DEF9FF00450025C026E6B
:103EE00005500358036E12009F0E046EFF0E056E00
:103EF00002C006F003C007F0045006260550072252
:103F000007500AE11A0E065CD8A089EF9FF08CEFEB
:103F10009FF0010E8DEF9FF0000E026E036A1200FB
:103F2000BF0E046EFF0E056E02C006F003C007F060
:103F3000045006260550072207500AE11A0E065CB7
:103F4000D8A0A5EF9FF0A8EF9FF0010EA9EF9FF07A
:103F5000000E026E036A1200D00E046EFF0E056E94
:103F600002C006F003C007F00450062605500722E1
:103F700007500AE10A0E065CD8A0C1EF9FF0C4EF1B
:103F80009FF0010EC5EF9FF0000E026E036A120053
:103F90000C6E0CC002F0036A000E056E0A0E046E71
:103FA000E7EC98F002C00AF003C00BF00CC002F07E
:103FB000036A000E056E0A0E046E08EC97F00250BC
:103FC000100DF3500A2412003D01799560000BF0AA
:103FD0006EFD000E6C6F738B79A5F1EF9FF0F3EF20
:103FE0009FF0ECEF9FF074ABF8EF9FF0FBEF9FF0CA
:103FF000010EFCEF9FF0000E12003901A3A903EFA0
:10400000A0F005EFA0F0FDEF9FF00D0E3D01EA6F6F
:104010003901A3A90EEFA0F010EFA0F008EFA0F077
:104020000A0E3D01EA6F1200000E036E000E026ED2
:1040300000F0024A032A03BE27EFA0F0035009E173
:10404000A00E025CD8A027EFA0F029EFA0F018EF97
:10405000A0F01200025004026F00CCFF06F06F00C7
:10406000D0FF07F002500502F35007260350040268
:10407000F350072606C002F007C003F0120010C07C
:1040800002F011C003F057EC9FF002501024066EAE
:1040900003501120076E12C008F013C009F064EC41
:1040A0009CF012006F0060FF01F00001784B792B4B
:1040B0009E81660EB76E7C0EB66E3901A39F6000BE
:1040C00007F0D8FF1100026E67EFA0F000F0390191
:1040D000A3A96DEFA0F06FEFA0F066EFA0F0600075
:1040E0000BF0EAFD1200800E3D01746F000E756F3B
:1040F000030E7B6F040E736F000E796F000E766FE8
:10410000738F1200106E0DC008F010508CEC98F0F8
:104110000EC006F00FC007F001EC9DF01200106E0B
:104120000DC008F010508CEC98F00EC006F00FC0D7
:1041300007F0B5EC9AF012003D0179A5A2EFA0F0CE
:10414000A4EFA0F09CEFA0F079957991788512000A
:10415000036E03C002F00F0E021603380F0B0A0D98
:10416000F35002241200140030304830304D30300B
:0441700053001200E6
:020000040020DA
:10000000FF0FFF0FFF0FFF0FFF0FFF0FFF0FFF0F80
:020000040030CA
:0A0000008CD5FFF78DCFFFDFFFFF67
:00000001FF
